:100000000C94AE030C94CB030C94E6030C94CB033A
:100010000C94CB030C94CB030C94FF1F0C94CB03D8
:100020000C94CB030C94CB030C94CB030C94CB0318
:100030000C94CB030C94CB030C9487200C94CB032F
:100040000C94CB030C94CB030C94CB030C94CB03F8
:100050000C94CB030C94CB030C94CB030C94CB03E8
:100060000C94CB030C94CB0379077907A507A5075C
:1000700014083208520952093D08D608E708E70873
:10008000506C6169642D506164202F2F2F2F2F2F0A
:100090002F2F2F2F2F005F006000610054005C00A5
:1000A0005D005E00550059005A005B00560062007A
:1000B00063006700570000AE00AF00DA0281FFD98D
:1000C000F1DB20A4A62EAF00A0C000A1C800AED5D1
:1000D00080A81FD300408D14200007087F08070068
:1000E0003E5B4F5B3E003E6B4F6B3E001C3E7C3EDA
:1000F0001C00183C7E3C18001C577D571C001C5EE1
:100100007F5E1C0000183C180000FFE7C3E7FF00FB
:10011000001824180000FFE7DBE7FF0030483A062C
:100120000E00262979292600407F05050700407F1B
:1001300005253F005A3CE73C5A007F3E1C1C080046
:10014000081C1C3E7F0014227F2214005F5F005FAA
:100150005F0006097F017F00006689956A00606084
:100160006060600094A2FFA2940008047E0408006E
:1001700010207E20100008082A1C0800081C2A08ED
:1001800008001E10101010000C1E0C1E0C00303841
:100190003E383000060E3E0E060000000000000053
:1001A00000005F000000000700070000147F147FBC
:1001B0001400242A7F2A120023130864620036499F
:1001C00056205000000807030000001C22410000D8
:1001D0000041221C00002A1C7F1C2A0008083E083F
:1001E00008000080703000000808080808000000BF
:1001F000606000002010080402003E5149453E00A6
:1002000000427F4000007249494946002141494D62
:1002100033001814127F10002745454539003C4A29
:100220004949310041211109070036494949360041
:10023000464949291E000000140000000040340017
:10024000000000081422410014141414140000418A
:10025000221408000201590906003E415D594E0072
:100260007C1211127C007F49494936003E414141D0
:1002700022007F4141413E007F49494941007F09B9
:10028000090901003E41415173007F0808087F00C1
:1002900000417F4100002040413F01007F081422BF
:1002A00041007F40404040007F021C027F007F04ED
:1002B00008107F003E4141413E007F0909090600C8
:1002C0003E4151215E007F091929460026494949CE
:1002D000320003017F0103003F4040403F001F20E8
:1002E00040201F003F4038403F0063140814630063
:1002F0000304780403006159494D4300007F4141E4
:100300004100020408102000004141417F00040226
:100310000102040040404040400000030708000084
:100320002054547840007F284444380038444444E2
:100330002800384444287F003854545418000008DA
:100340007E09020018A4A49C78007F0804047800A9
:1003500000447D4000002040403D00007F102844C4
:10036000000000417F4000007C04780478007C0895
:1003700004047800384444443800FC18242418004D
:1003800018242418FC007C08040408004854545421
:10039000240004043F4424003C4040207C001C20F6
:1003A00040201C003C4030403C00442810284400C1
:1003B0004C9090907C004464544C440000083641BA
:1003C0000000000077000000004136080000020134
:1003D000020402003C2623263C000000000000002E
:1003E000404040F0F8F8FF38FFF8F83FF8F8FF38E1
:1003F000FFF8F8F040404000000000000080C0C05E
:10040000C0800000C0C08000000080C0C000C0C02C
:10041000000080C0C00000000000C0C0C0C0C0001C
:10042000C0C000000000000000000000000000004C
:1004300000000000000000000000000000000000BC
:1004400000000000000000000000000000000000AC
:10045000000000000000000000C0F0F8FC3E1E0696
:10046000010000007F4141417F007F4141417F0009
:100470000080C0E07E5B4F5BFEC00000C000DCD7A8
:10048000DEDEDED7DC00C00000000000000000005F
:10049000000000000000000000000000000000005C
:1004A000494949FFFFFFFFE0DFBFBF00BFBFDFE0FB
:1004B000FFFFFFFF49494900000000001F3F606047
:1004C000E0BF1F007F7F071E381E077F7F007F7FF2
:1004D0000E1F3B716000000000007F7F0C0C0C00C1
:1004E0007E7E007F7E0303007F7E03037E7E030308
:1004F0007F7E000F3E703C063C703E0F00327B4911
:10050000493F7E007F7E0303001E3F69696F26001E
:10051000000000000000000000030F1F3F3C787047
:10052000600000007F4141417F007F4141417F00E9
:10053000307B7F7830202030787F3B0003000F7FB6
:100540000F0F0F7F0F0003000000000000000000ED
:10055000000000000000000000000000000000009B
:10056000010101070F0F7F0F7F0F0F7E0F0F7F0F0E
:100570007F0F0F07010101000000000000000000D4
:100580000001010000000000000000000000000069
:10059000000000000000000000000000000000005B
:1005A000000000000000000000000000000000004B
:1005B000000000000000000000000000000000003B
:1005C000000000000000000000000000000000002B
:1005D000000000000000000000000000000000001B
:1005E000000000000000000000000000000000000B
:1005F00000000000000000000000000000000000FB
:1006000000000000000000000000000000000000EA
:100610000000000000000000000009023B00020191
:1006200000A03209040000010301010009210101B9
:1006300000012240000705810308000109040100B0
:100640000103000000092101010001227B000705D0
:100650008303080001120110010000000883795093
:10066000500300010200011E0350006C006100698C
:100670000064002D005000610064002000520065FD
:100680000076003300000014034B0065007900631E
:100690000061007000730073007300000004030920
:1006A0000405010902A10185020901A1000509193A
:1006B0000129081500250195087501810205010928
:1006C0003009311581257F95027508810609381595
:1006D00081257F950175088106050C0A3802158170
:1006E000257F950175088106C0C005010980A1011B
:1006F000850319012AB700150126B7009501751069
:100700008100C0050C0901A101850419012AA0027C
:10071000150126A002950175108100C0050109068A
:10072000A101050719E029E71500250195087501C4
:1007300081029501750881030507190029FF15003D
:1007400026FF009506750881000508190129059501
:100750000575019102950175039103C011241FBE17
:10076000CFEFD8E0DEBFCDBF11E0A0E0B1E0E6EC16
:10077000F8E402C005900D92AC3AB107D9F725E034
:10078000ACEAB1E001C01D92AF36B207E1F70E94BA
:1007900044150C9461240C940000A82FB92F80E01C
:1007A00090E041E050EA609530E009C02D91822749
:1007B0009795879510F084279527305EC8F36F5F73
:1007C000A8F30895EADF8D939D930895CF93CFB753
:1007D000CF93DF93C3954B9BE9F74B9B10C04B9B8B
:1007E0000EC04B9B0CC04B9B0AC04B9B08C04B9B45
:1007F00006C0C0914605C395C09346058EC06F9351
:10080000C0914505DD27C35BDA4F2F9365E54B9B10
:1008100003C02F916F91E1CF0F931F934F9320E06F
:1008200040E15F9309B10C7003FB27F93F9350E05F
:100830003BE039C01C7040642F77012F5F5F1EC002
:10084000406819B11C702F7752501FC0406409B125
:100850002F770C70D1F15F5F00C023C0406219B1E7
:100860002F771C7091F15F5F00C025C00C701027BE
:10087000515012F45D5F0000115027952C3F19B1C3
:10088000C8F61C700127015027952C3FC8F6422757
:10089000499309B10C7010274F73115027952C3FC5
:1008A000A8F64695469519B11C7079F001270150BC
:1008B00027952C3F98F66B5A60F3315009B1B0F68A
:1008C00000C012E01CBB00271CC03B503195C31B6D
:1008D000D04012E01CBB0881033C21F10B3411F124
:1008E000209142051981110F1213EDCF4A81441F47
:1008F000093679F10D3211F0013E29F74F7009F0F8
:10090000042F00934B053F915F914F911F910F91E1
:100910002F916F91CCB3C1FD5DCFDF91CF91CFBF50
:10092000CF91189520914B05222369F31091490529
:10093000112309F049C034300AF448C03093490506
:1009400020934405109145053BE0311B309345054C
:100950003DC0009149050130BCF50AE54F7049F4EE
:100960003091200134FD33C000932001CFE1D5E068
:1009700032C0433059F0443091F030912A0534FDB3
:1009800026C000932A05CBE2D5E025C0309163054F
:1009900034FD1DC000936305C4E6D5E01CC0309152
:1009A000360534FD14C000933605C7E3D5E013C007
:1009B000052710E000C000000BB91AC0052710E0A1
:1009C000221F1DC010E021C04AE502C032ED432FB6
:1009D000C4E1D0E032E01AB11C605B9A0BB11AB9E5
:1009E0005CE020E865E320FF05270BB92795179504
:1009F0001C3FF0F66695B8F7B1F720FF05270BB955
:100A0000279517951C3FD0F62795179517FF0527B3
:100A100000001C3F0BB9B0F629913A9519F7037FF6
:100A200010914A05110FC651D0400BB911F0109327
:100A3000420512E01CBB08601AB1137F402F437FB0
:100A400054E05A95F1F70BB91AB94BB95CCF60E095
:100A500080E890E00E94541980E00895811106C05A
:100A6000662311F08CE619C08DE617C0813031F491
:100A7000662311F08EE611C08FE60FC0823031F48C
:100A8000662311F080E709C081E707C0833039F49D
:100A9000662311F082E701C083E70E94270781E007
:100AA000089581E0089581E008950C945305089518
:100AB0000C9457051F93CF93DF9300D000D01F9263
:100AC000CDB7DEB749835A836B833091AF018981FB
:100AD0009A81311114C0662359F0222349F00E94F3
:100AE0008D0B182F682F89819A810E94380B03C0C3
:100AF0000E94620B182F69817A81812F04C00E94A5
:100B00008D0B69817A810F900F900F900F900F904D
:100B1000DF91CF911F910C94CF12FC01262F4081C1
:100B200051816281738184810C945A0581E008951A
:100B3000CF93DF93EC0160E00E948D05BE01DF9151
:100B4000CF910C9458050C9413140C940F14089521
:100B50000E94E2090E94A7052FEF84E39CE0215048
:100B600080409040E1F700C000000C94AD200F934E
:100B70001F93CF93DF938C0161E00E948D05EC0100
:100B8000B8010E9455058823F1F1B801CE010E94F9
:100B9000D61D8823C1F1B801CE010E94C71A88234F
:100BA00091F1B801CE010E94321D882361F1F80154
:100BB0008281882309F1CB358DE5D807C1F050F447
:100BC000C115FCE5DF0781F0CF3DDC45A9F40E94AB
:100BD000C41019C0CC35EDE5DE0761F0CD35DD453B
:100BE00059F40E94071008C00E94A8050CC00E947A
:100BF000101002C00E941310C801DF91CF911F9105
:100C00000F910C94510580E0DF91CF911F910F91CE
:100C100008950E94E21F0E9424060C947D1A0E94EF
:100C200027060C94E81F08950C94130681E008959C
:100C30000C9416060895CF93C82F0E9414068C2F8B
:100C40000E941806CF91089580E00C941B060E9424
:100C5000411F0C941B060E94411F9091AE01891701
:100C600021F08093AE010C941B060895CF93DF937F
:100C7000CDB7DEB72B970FB6F894DEBF0FBECDBF52
:100C80004F83588769877A878B8761110E94530F3A
:100C90009E012F5F3F4F86E0F90111928A95E9F797
:100CA00085E0FE013796D90101900D928A95E1F712
:100CB00089819A814C815D81452B31F09F3F31F4D0
:100CC00091E08F3F19F403C091E001C090E090FFE4
:100CD00009C049815A816B817C818D819E810E94EE
:100CE000740E05C0C9010E9496058111F2CF2B96A2
:100CF0000FB6F894DEBF0FBECDBFDF91CF91089540
:100D0000FC01808191810E94CF0B0895CF938823AD
:100D100009F450C0C82F8CEF8C0F813AD0F46C2F9F
:100D200080910201909103010E949E1F882349F047
:100D30006C2F80910201909103010E94D61F0E94A6
:100D4000750F6C2F80910201909103010E94D41FB6
:100D50000CC080E28C0F883058F4C77081E001C06D
:100D6000880FCA95EAF70E94360FCF910C94750F41
:100D7000EBE5EC0FE33040F4F0E0E15BFE4F808107
:100D800090E0CF910C94661FE8E5EC0FE73150F44A
:100D9000F0E0EE0FFF1FEF5DFE4F80819181CF915C
:100DA0000C947C1FCD3E30F08C2F0E94C915CF9142
:100DB0000C949B16CF910895882389F19CEF980F8E
:100DC000913A40F4682F80910201909103010E94B2
:100DD000D61F0DC090E2980F983058F4877091E0BC
:100DE00001C0990F8A95EAF7892F0E943C0F0C9455
:100DF000750F9BE5980F933020F480E090E00C9401
:100E0000661F98E5980F973120F480E090E00C94ED
:100E10007C1F8D3E20F00E9424160C949B16089592
:100E20001F93CF93DF93182FEB010E948606209724
:100E300041F08FE99FE00197F1F700C00000219792
:100E4000F6CF812FDF91CF911F910C94DC0689336F
:100E500019F06CE370E002C060E570E00C941007DC
:100E6000882321F00E94360F0C94750F0895882373
:100E700021F00E943C0F0C94750F0895CF92DF92E1
:100E8000EF92FF920F931F93CF93DF937C01D62FA6
:100E9000C72FFC011281058102950F700E942C0F53
:100EA0008823B9F01123A9F08C2F807F803421F0A2
:100EB00080E28D0F883068F080910C0382FD09C0BC
:100EC00082E00E94D50F0E942C0F91E0D82ED926E7
:100ED00001C0D12CCC2EC2948FE0C8228C2D90E082
:100EE0008C30910508F0DEC1FC01EC5CFF4F0C94E6
:100EF00003248C2F807FCF70882311F0C295C07F90
:100F0000112399F0CC2309F4B1C180E28D0F883010
:100F100010F0D11104C08C2F0E94360F03C08C2F0B
:100F20000E94460F0E94750FA1C18D2F0E94DC0602
:100F3000CC2309F4B7C180E28D0F883038F1DD236E
:100F400029F18C2F0E944C0F24C08C2F807FCF70F2
:100F5000803211F0C295C07FDD2319F0D130A1F1AC
:100F60003DC080910C0382FF17C0112349F0CC23B0
:100F700029F08C2F0E94360F0E94750F80E077C1F8
:100F800080E00E94DC06CC2309F48CC18C2F0E94E7
:100F90003C0F0E94750F86C1112371F0002341F0B0
:100FA000013031F40E94560F8C2B0E945E0F7AC1E3
:100FB0000E94560F8C2B1DC0002319F0013009F43C
:100FC00071C10E946B0F2CC0112321F0063008F074
:100FD00069C10EC0053008F065C122C0112361F05F
:100FE000002331F0F701858180FF40C18F70858338
:100FF0008C2F0E94300756C1002391F0D93341F461
:10100000FFEF07EE13E0F15000401040E1F745C15B
:101010002FEF3DEE82E0215030408040E1F73DC1AE
:101020008C2F0E9437073EC18C2F86958695837042
:1010300019F0813061F036C1112321F08D2F9C2FE2
:10104000937002C080E090E00E94661F33C11123BC
:1010500021F08D2F9C2F937002C080E090E00E94C1
:101060007C1F28C18D2F112319F00E94C91502C0C1
:101070000E9424160E949B161DC18C2F837009F0BC
:1010800047C0111113C12D2F229526952770220FCD
:10109000220F6D2F6F70862F90E0A0E0B0E0022E3F
:1010A00004C0880F991FAA1FBB1F0A94D2F7D4FF50
:1010B00010C04FE050E060E070E004C0440F551FE6
:1010C000661F771F2A95D2F74095509560957095C9
:1010D00003C040E050E0BA01C695C695C3708A01CE
:1010E0009B01082B192B2A2B3B2BC901B801C230BD
:1010F00049F058F4C13019F00E944E0AD7C00E943E
:101100003C0AD4C00E94600AD1C00E943A0ACEC0F4
:10111000112319F08C2F817001C08695882309F462
:10112000C5C02D2F229526952770220F220F6D2FD7
:101130006F70862F90E0A0E0B0E0022E04C0880F10
:10114000991FAA1FBB1F0A94D2F7D4FF10C04FE00B
:1011500050E060E070E004C0440F551F661F771F29
:101160002A95D2F7409550956095709503C040E060
:1011700050E0BA01C695C695C3708A019B01082B41
:10118000192B2A2B3B2BC901B801C23049F058F466
:10119000C13019F00E94130B89C00E94010B86C058
:1011A0000E94250B83C00E94740A80C0CF70112357
:1011B00039F08C2F0E949A0A8D2F0E94300776C03A
:1011C0008D2F0E9437078C2F0E94BB0A6FC0D23F21
:1011D00021F128F4D03F41F0D13FC1F043C0D33FCB
:1011E00019F1D43F79F03EC0112341F0053008F0E9
:1011F00059C08C2F8F710E94E00A54C0063008F04D
:1012000051C0F7CF80910C0382FF18C0112339F031
:101210008C2F8F710E949A0A45C01123C9F38C2F1D
:101220008F710E94BB0A3EC0112329F08C2F8F7151
:101230000E94850A37C00E94800A34C0112349F0F9
:10124000CF718C2F0E949A0A63E08C2F0E94BA0FF4
:1012500029C081E00E94D50F023020F182E00E9477
:10126000D50F20C0112331F0002391F28D2F0E9461
:10127000860618C0002399F2D93341F41FEF27EEF8
:1012800033E0115020403040E1F707C08FEF9DEE72
:10129000E2E081509040E040E1F700C000008D2F77
:1012A0000E94DC0688EF8C0D843020F40E94411FE0
:1012B0000E941B06DD20C9F00E94280F80FD15C08A
:1012C000F70112820E94220F0E949A0AC7010E940F
:1012D00096090E94220FDF91CF911F910F91FF90ED
:1012E000EF90DF90CF900C94BB0ADF91CF911F91CC
:1012F0000F91FF90EF90DF90CF9008950F931F9381
:10130000CF93DF93EC01688179818A810E94DA0BA7
:101310008C010E94370B0E94280AB801CE010E945E
:101320003E07DF91CF911F910F910895CF93DF93E7
:10133000EC01988189812B813C81232B31F08F3FF7
:1013400031F481E09F3F19F403C081E001C080E0E7
:1013500080FD1DC0CE010E94B705811110C00E9402
:101360002C0F8823A1F08A81882389F080910C03B7
:1013700082FD0DC082E0DF91CF910C94D50FCE019C
:101380000E947E09CE01DF91CF910C949805DF91E8
:10139000CF91089580E090E00E94661F80E090E089
:1013A0000E947C1F0E94530F0E94750F0E94CC1751
:1013B0000C949B1680910201909103010E94D81F0A
:1013C0000C94CA090E94430F0C94DA0992959F70FD
:1013D000963079F010F4925001C09A50923068F42F
:1013E000803F69F018F4883E40F409C0843F29F436
:1013F00006C0883E20F0813F11F080E0089581E032
:101400000895FC01808191810E94CF0B0E94E60922
:101410000895CF93DF9300D000D01F92CDB7DEB7F1
:101420000F900F900F900F900F90DF91CF91089534
:10143000CF93DF9300D000D000D0CDB7DEB7269693
:101440000FB6F894DEBF0FBECDBFDF91CF910895E8
:10145000089508950C94290A0C942A0A0E942C0AD3
:101460006093BE017093BF018093C0019093C1014E
:101470000C94CA090C942E0A0F931F930091BE017D
:101480001091BF012091C0013091C101602B712BDF
:10149000822B932B1F910F910C942E0A0F931F9365
:1014A0000091BE011091BF012091C0013091C10196
:1014B00060237123822393231F910F910C942E0A92
:1014C0000F931F930091BE011091BF012091C001A5
:1014D0003091C10160277127822793271F910F91B7
:1014E0000C942E0A0C94290A0E94720A6093BA0185
:1014F0007093BB018093BC019093BD010C94CA0909
:1015000060E070E0CB010C94740A0F931F9341E0EC
:1015100050E060E070E08A019B0104C0000F111FE1
:10152000221F331F8A95D2F7C901B8011F910F916D
:101530000C94740A0F931F9341E050E060E070E058
:1015400004C0440F551F661F771F8A95D2F78091FC
:10155000BA019091BB01A091BC01B091BD018A017B
:101560009B01082B192B2A2B3B2BC901B8011F917A
:101570000F910C94740A0F931F9341E050E060E0C8
:1015800070E004C0440F551F661F771F8A95D2F77D
:1015900040955095609570958091BA019091BB01EE
:1015A000A091BC01B091BD018A019B0108231923C0
:1015B0002A233B23C901B8011F910F910C94740A8F
:1015C0000F931F9341E050E060E070E004C0440FCF
:1015D000551F661F771F8A95D2F78091BA019091A7
:1015E000BB01A091BC01B091BD018A019B010827FC
:1015F00019272A273B27C901B8011F910F910C9485
:10160000740A0F931F930091BA011091BB012091AE
:10161000BC013091BD01602B712B822B932B1F914C
:101620000F910C94740A0F931F930091BA011091BB
:10163000BB012091BC013091BD0160237123822345
:1016400093231F910F910C94740A0F931F93009191
:10165000BA011091BB012091BC013091BD016027FE
:101660007127822793271F910F910C94740A089574
:10167000990F990F890FE82FE695E695E695877003
:1016800051E001C0550F8A95EAF785E0E89FF00127
:101690001124E055FE4F20E030E070E04081CB01A6
:1016A000022E02C0969587950A94E2F78170819583
:1016B00084278523842781932F5F3F4F2530310571
:1016C00069F70895990F990F890F682F66956695A8
:1016D0006695982F977085E0689FB001112440E0CF
:1016E00050E080E0FB01E40FF51FE055FE4F208144
:1016F00030E0092E02C0369527950A94E2F7217052
:101700003327042E01C0220F0A94EAF7822B4F5F81
:101710005F4F4530510531F70895BF92CF92DF9268
:10172000EF92FF920F931F93CF93DF938C01C090A2
:10173000BA01D090BB01E090BC01F090BD01809156
:10174000BE019091BF01A091C001B091C101C82A12
:10175000D92AEA2AFB2ACFE1D0E0D701C6010C2E14
:1017600004C0B695A795979587950A94D2F780FD02
:1017700004C0219790F7B12C07C0BC2EB8018C2F64
:101780000E94E3120197A9F38B2DDF91CF911F9156
:101790000F91FF90EF90DF90CF90BF900895CF937F
:1017A000DF93EC010E948D0BBE010E94E312DF91DA
:1017B000CF9108951F93CF93DF93EB019091AF01E9
:1017C000992321F0CB010E94CF0B13C0882349F04D
:1017D000CB010E948D0B182F682FCE010E94380B71
:1017E00004C0CB010E94620B182FBE01812F0E9402
:1017F000E312DF91CF911F9108951F93CF93DF9351
:10180000C091C20116E08091C301C81799F0D0E0E1
:101810001C9FF0011D9FF00D1124EC53FE4F4081E1
:10182000518162817381848195810E94180A219679
:10183000C770E9CFDF91CF911F9108954091F401D6
:101840005091F5016091F6017091F7018091F801D6
:101850009091F9010C94180AEF92FF920F931F9345
:10186000CF93DF938091F90182958F7009F065C065
:101870008091F601882309F460C08091C201F09044
:10188000C3011091F4010091F5016091F70170918D
:10189000F80191E01F3F09F090E0C0910001D09164
:1018A0000101292F96E0E92E8F1509F446C0611534
:1018B000710521F00F3F21F030E003C031E001C09D
:1018C000322F90E030FD36C0E89EF001E99EF00D29
:1018D0001124DF01AC53BE4F11963C911197301388
:1018E00029C03C91311326C012963C9112973111B8
:1018F00021C013964D915C911497461B570B4C17C2
:101900005D07C0F48091F9018F7080618093F901C7
:10191000E753FE4F80818F708061808384EF91E078
:101920000E949609DF91CF911F910F91FF90EF9048
:101930000C94FD0B01968770B7CFDF91CF911F916B
:101940000F91FF90EF9008959F92AF92BF92CF9228
:10195000DF92EF92FF920F931F93CF93DF93CDB758
:10196000DEB761970FB6F894DEBF0FBECDBF8C0116
:1019700085E0F801DE011D9601900D928A95E1F750
:10198000D8011296EC909091F401E091F50120912C
:10199000F7013091F8012115310531F0EF3F31F4B5
:1019A00081E09F3F19F403C081E001C080E0B82FBF
:1019B000B1709B2E80FD47C1D8014C9111965C916E
:1019C00011971396AD90BC90149784EFC82E81E0C8
:1019D000D82EF090F601B501621B730B2091000127
:1019E00030910101FF2009F4D9C08091F9016217FB
:1019F000730708F095C0282F207F09F052C05E13AE
:101A000013C0491311C0FE2CE1100EC08F7080610D
:101A10008093F9010E941E0CC6010E9496098091D4
:101A2000F901F80185834DC1AB2831F05F3F31F4F6
:101A300081E04F3F19F403C081E001C080E080FDE8
:101A400003C081E08E2502C080E090E0F82FF170A5
:101A5000FF2E80FF1CC08091C2012091C30136E09F
:101A6000821709F40BC190E0389FF001399FF00D07
:101A70001124EC53FE4F6181561306C0608146135A
:101A800003C06281E61203C001968770E9CFFE2C85
:101A9000EE2009F416C18091F90181608093F9016B
:101AA00054C05E1306C0491304C0E11002C0F8011F
:101AB00099C0C8010E94010A882361F1EE2051F10A
:101AC0002091F901822F82958F7090E0029774F037
:101AD0008091F4019091F50198878F831986BB86D8
:101AE000AA862C87CE0107960E94960986E0F80107
:101AF000A4EFB1E001900D928A95E1F70E942C0CC1
:101B00000E941E0C0AC05E1711F1C8010E94010A52
:101B100081112CC0C8010E949609FF24F394D1C002
:101B2000282F207F81F77A2DB98AA88A6E2D89897E
:101B30000E94090A84EF91E00E94960986E0D6018E
:101B40001D928A95E9F70E941E0CF12CBAC0491328
:101B5000DCCFE110DACFF8018583C8010E94960935
:101B600086E0D6011D928A95E9F7ABC0EE2091F28E
:101B70002091F901822F82958F7090E002970CF4EA
:101B8000B5CF8091F4019091F5019A8389831B82EE
:101B9000BD82AC822E83CE010196A6CF6217730759
:101BA00008F044C0FE2CEE2009F4B4CF5E1330C020
:101BB00049132EC02091F90120FD21C0822F82956A
:101BC0008F70482F50E041155105C9F0F801258369
:101BD0004F30510541F08F5F982F9295907F822F63
:101BE0008F70892B8583C8010E94960986E0F801D1
:101BF000A4EFB1E001900D928A95E1F73CC086E038
:101C0000F801A4EFB1E001900D928A95E1F759C077
:101C1000C8010E94010A811169CF8091F901816098
:101C20008093F901C8010E9496094BC07A2DB98AA8
:101C3000A88A6E2D89890E94090A86E0D6011D9224
:101C40008A95E9F718C0EE2009F464CFC8010E9414
:101C5000010AF82E882309F45DCF86E0F801A4EF8D
:101C6000B1E001900D928A95E1F784EF91E00E9436
:101C700080060E942C0C0E941E0C23C04D875E879C
:101C80008D859E850E94CF0B292F22952F702230A3
:101C900028F49F7039F0811105C00BC0243028F45E
:101CA0009F7049F4805E883020F0C8010E94960938
:101CB0009F2CF92C06C0D80115969C91907F91F726
:101CC000F8CF8F2D61960FB6F894DEBF0FBECDBF53
:101CD000DF91CF911F910F91FF90EF90DF90CF9008
:101CE000BF90AF909F9008951F93CF93DF93CDB790
:101CF000DEB72C970FB6F894DEBF0FBECDBF4F8373
:101D0000588769877A878B879C87CE0107960E94C0
:101D1000A40C8823D1F09F8188852A853B85232BBD
:101D200031F08F3F31F481E09F3F19F403C081E02F
:101D300001C080E080FD47C04F81588569857A8564
:101D40008B859C850E94180A3EC086E0FE0137966E
:101D5000DE01119601900D928A95E1F7FF81E885E9
:101D60006A857B856115710531F0EF3F31F481E0C3
:101D7000FF3F19F403C081E001C080E080FD23C073
:101D80002091C30130E0C9010196877099274091E5
:101D9000C20150E084179507F1F1F983EA837D834E
:101DA0006C8396E0929FD001939FB00D1124AC53A9
:101DB000BE4FFE01319601900D929A95E1F7809306
:101DC000C3010E94FD0B16E08091C2019091C301F6
:101DD000891771F1189FC00111248C539E4F0E94E6
:101DE000A40C882329F1E091C2011E9FF001112467
:101DF000EC53FE4F408151816281738184819581D2
:101E00000E94180A8091C20190E00196877099277C
:101E10008093C201D9CF0E94E2091092C3011092AF
:101E2000C201E4EFF1E086E0DF011D928A95E9F757
:101E30002C960FB6F894DEBF0FBECDBFDF91CF91C9
:101E40001F91089580910202859585958595089545
:101E5000809102028770089590910202977081E04C
:101E600009F480E0089580910D02089590910D028B
:101E7000892B80930D020895809590910D028923FE
:101E800080930D02089510920D02089590910C0216
:101E9000892B80930C020895809590910C028923E0
:101EA00080930C02089510920C0208958091030211
:101EB000089508950C94590F0C945A0F90910C03A7
:101EC00092FD08C090910302981721F080930302BD
:101ED0000C945C0F089580910302882329F01092DE
:101EE000030280E00C945C0F0895CF93DF93E091A0
:101EF0000201F091030180910D028083E0910201C3
:101F0000F0910301908180910C02892B8083809154
:101F10000302882381F0E0910201F0910301908196
:101F2000892B808380910201909103010E94921F6E
:101F300081110E946B0FC0910201D091030148E012
:101F400050E06AEF71E0CE010E941224892B69F003
:101F500088E0FE01AAEFB1E001900D928A95E1F7C9
:101F6000CE01DF91CF910C944D1FDF91CF91089559
:101F70000C94590F90910C0392FD10C098E0899F2A
:101F800090011124262B209302020E949A0A80912C
:101F900002028595859585950C94B80F0C949A0A44
:101FA0001092020280E00C94B80F209102028095FA
:101FB000822380930202982F977099F430E0482F83
:101FC000082E000C550B2417350759F090910C037F
:101FD00092FD07C08595859585950E94BB0A0C9456
:101FE000D00F089590910C0392FB222720F9281717
:101FF00069F080FB92F990930C0380910B03909110
:102000000C030E94401082E00C94D50F089580913B
:102010000C0382FB882780F991E089270C94F20F4A
:1020200081E00C94F20F80E00C94F20F6FEF7FEFE1
:1020300080E090E00C944B2480E090E00E94272404
:1020400021E0893E9E4F09F020E0822F089582E032
:1020500090E00C941F2483E090E00C941F24CF9315
:1020600084E090E00E941F24C82F82E290E00E944A
:102070001F242C2F30E0A901582BCA01CF910895BD
:10208000CF93C92F682F84E090E00E942D246C2FFD
:1020900082E290E0CF910C942D24AB01BC018FE043
:1020A00090E00C943F24AB01BC0183E190E00C94E0
:1020B0003F2460E070E0CB010C94531060E070E0CE
:1020C000CB010E944D100C94591069EE7EEF80E018
:1020D00090E00E944B2460E082E090E00E942D247A
:1020E00060E083E090E00E942D241092BE011092E7
:1020F000BF011092C0011092C10160E084E090E045
:102100000E942D2460E082E290E00E942D2460E095
:1021100085E090E00E942D2460E086E090E00E943F
:102120002D246FEF87E090E00E942D2440E050E0E6
:10213000BA0188E090E00E943F2460E08DE090E0EA
:102140000E942D2440E050E0BA0188E190E00E9416
:102150003F2460E087E190E00E942D2440E050E0C1
:10216000BA018CE190E00E943F2460E070E080E2E0
:1021700090E00E944B2440E050E0BA0188E190E0FA
:102180000E943F240C945E100C946510682F8EE022
:1021900090E00C942D240E946C2060931A0270939E
:1021A0001B0280931C0290931D0260931602709391
:1021B0001702809318029093190208950E946C20D0
:1021C00060931A0270931B0280931C0290931D026D
:1021D000609312027093130280931402909315027D
:1021E000089581E008950C94F11008950C94F51071
:1021F0000C94F5100C94F8100C94F5100C94FC1041
:102200000C94F5108FEB93E10E94371F0E94001190
:102210000C94FE100E94F6100C94F5100E94D91335
:102220000C941A060E9457200E94B0140E940E11AE
:1022300080E00E941B180E94181C0C94FA108F92C8
:102240009F92AF92BF92CF92DF92EF92FF920F9345
:102250001F93CF93DF93CDB7DEB72A970FB6F894CD
:10226000DEBF0FBECDBF0E94C514982E81110E9403
:10227000CB108EE0A82E82E0B82E00E010E0802E79
:10228000802F0E94FD13D82EF501C1905F01C82652
:10229000B1F40F5F1F4F0430110589F78FEF898369
:1022A0008A831B820E9460208160782F9D838C83AB
:1022B00049815A816B818D810E9436062FC08091A1
:1022C0001E0281FD0E940314E12CFF24F3948C2D47
:1022D0008F21F1F00E94F310882399F0EE828F8213
:1022E000DF2081E009F480E088870E94602081601F
:1022F000782F9A8789874E815F8168858A850E94B9
:102300003606F801E25FFD4F8081F826F08206C0B4
:10231000E394FF0CF4E0EF12DACFBBCF81E0911031
:1023200001C080E02A960FB6F894DEBF0FBECDBF85
:10233000DF91CF911F910F91FF90EF90DF90CF90A1
:10234000BF90AF909F908F900895CF93DF930E949E
:102350001F11D82F0E948D1CC82F81110E94DE10E2
:102360000E94991AD11101C0C1110E9459190E94ED
:10237000B916DF91CF910C942B06CF93DF930E9477
:10238000E812EC01811521E5920708F045C081159E
:1023900030E5930708F094C0883E910528F5803E0B
:1023A000910508F0F8C0883A910570F4853A9105D6
:1023B00008F07CC08130910509F475C008F4E8C0CC
:1023C000049708F0E8C0E4C08F3B910508F0E0C036
:1023D000C85AD0E0CC0FDD1FCE5ADE4F0990D8810D
:1023E000C02DCE019464D8C0811540E2940758F402
:1023F000811551E0950708F0CEC08D3E910508F497
:10240000C7C09065C9C0C11580E4D80708F4C0C032
:10241000DF70CE01906AC0C0811525E59207A8F44F
:10242000811534E5930708F095C0811543E59407BD
:1024300008F07BC0811552E5950708F061C0D82FE0
:10244000CC27CE01816F906AA7C0C11589E5D80756
:10245000A0F4C11528E5D20708F082C0C11536E501
:10246000D30708F095C08C2F0E947C138F7190E0E9
:10247000D82FCC27CE0190628FC0C1154AE5D40772
:1024800008F474C0CE0190568115904208F080C0C7
:102490008D2F8F710E947C13DD27D0628F71AE016A
:1024A000582BCA0179C081E090E076C0C55AD0E0CF
:1024B000C058DE4F8881C82FD0E0CE0190646CC038
:1024C00074E0969587957A95E1F7282F23703C2F35
:1024D000337081E090E002C0880F991F3A95E2F7CF
:1024E0009C68AC01522B9A019C2F9F7096959695F3
:1024F00050E2959FE0011124C9018C2B9D2B4CC00B
:102500008370992721E030E002C0220F331F8A95A3
:10251000E2F79C2F9695969580E2989FE001112412
:10252000C22BD32BCE019C6837C08370992721E042
:1025300030E002C0220F331F8A95E2F79C2F969558
:10254000969540E2949FE0011124C22BD32BCE013B
:102550009A6822C0D82FCC27CE01846F906A1CC005
:10256000DC2FCC27CE01806F906A16C08C2F8F7025
:102570000E947C1394E0D695C7959A95E1F7CF70A9
:10258000D0E0DC2FCC27D0699E01282BC90104C0E4
:1025900080E090E001C0CE01DF91CF910895E72F58
:1025A000F0E094E0899FE00DF11D1124EE0FFF1F74
:1025B000EE0FFF1FE60FF11DEE0FFF1FEA56FF4F54
:1025C0008591949108950E94CF120E94BD110895A3
:1025D0008238910569F1B0F48133910509F46DC039
:1025E00048F48932910509F463C08A32910509F4EF
:1025F00069C008958533910509F455C08933910563
:10260000B9F00895833E910569F138F4803E910553
:10261000B1F0823E910509F10895863E9105A9F138
:10262000873E9105B9F1843E910509F064C023C04D
:1026300020910B0320FD4FC021FD4DC008958091D6
:102640000B0380FD44C080910C0380FF44C0809147
:102650000B0384FD42C083EE4DC080910B0382FFCB
:1026600038C0F5CF80910B0382FD33C080910C03FD
:1026700080FD31C0ECCF80910C0381FF32C080918E
:102680000B0384FD2AC087EE35C080910B0383FFC6
:1026900026C0F5CF80910B0383FD21C080910C03F0
:1026A00081FD1FC0ECCF80910B0385FD1CC01DC0B8
:1026B00080910B0385FD19C016C080910B0386FD28
:1026C00016C017C080910B0386FD13C010C089E3AC
:1026D00011C082EE0FC080EE0DC080E00BC086EE10
:1026E00009C084EE07C089E205C085E303C08AE221
:1026F00001C081E390E0089590910B0392FF0DC01B
:10270000282F2871283019F4877F846006C0282F6D
:102710002471243011F48B7F886093FF0DC0282F23
:102720002871283119F4877E846106C0282F24710E
:10273000243111F48B7E886120910C0320FF0DC0A1
:10274000382F3871383019F4877F816006C0382FF0
:102750003171313011F48E7F886021FF0DC0282F38
:102760002871283119F4877E816106C0282F2171D4
:10277000213111F48E7E886194FD877E089580E07A
:1027800008950C9416100E94C5148FE39CE90197DC
:10279000F1F700C000000E94C51480E00E94FD1304
:1027A00080FF04C00E94C1130C94AD2008950C94C6
:1027B000C3130E941C10811102C00E94C4100E9409
:1027C000271080931E020E942F1090930C03809379
:1027D0000B030E94D7130E942B10682F70E080E03B
:1027E00090E00E943A0A6091BA017091BB01809119
:1027F000BC019091BD010C94720AE82FF0E0EF5EED
:10280000FC4F80810895089580EA8A95F1F7089534
:1028100000C008950C94041408950C940C140C94A6
:102820000D140C940C140C941114F894E82FE295E8
:10283000EF70F0E031A1282F2F7081E090E001C00F
:10284000880F2A95EAF7982F9095932391A392A148
:10285000892B82A3789408950F931F93CF93DF93CE
:10286000C7E8D1E089918F3F11F00E94151481E0F3
:10287000CB38D807B9F7C3E8D1E007E811E0899170
:102880008F3F11F00E9415140C171D07C1F7DF913F
:10289000CF911F910F910895CF92DF92EF92FF9207
:1028A0000F931F93CF93DF938C01C62FD0E0CE01FF
:1028B00089579E4F7C01FC0190819F3F09F447C0DE
:1028C000D62EF894E92FE295EF70F0E081A19F7089
:1028D00021E030E001C0220F9A95EAF7822B81A314
:1028E00082A12095282322A378940E940814E3E86B
:1028F000F1E047E851E031E0C12C21912F3F89F010
:10290000A22FA295AF70B0E090968C9190E02F70BE
:1029100002C0959587952A95E2F780FD02C0832F26
:1029200001C080E0C82A330F4E175F0731F7F70167
:1029300080818F3F11F00E94151461E0C11001C029
:1029400060E08D2D0E940A14C00FD11FC882DF9154
:10295000CF911F910F91FF90EF90DF90CF9008954E
:102960000E942C1484E0E1E1F3E0DF01982F1D9236
:102970009A95E9F7EDE0F3E0DF011D928A95E9F71A
:1029800084E00E9407150C94A3051F93CF93DF9357
:1029900000D000D0CDB7DEB719821A821B821C820C
:1029A00010E0612FCE0101960E944C141F5F14307D
:1029B000C1F744E050E0BE016F5F7F4F8DE093E0D0
:1029C0000E94122411E0009709F410E0892B61F0B5
:1029D00089819A81AB81BC8180930D0390930E0312
:1029E000A0930F03B0931003212F44E061E173E043
:1029F0008DE093E00E9408150E94A505812F0F909D
:102A00000F900F900F90DF91CF911F91089508952F
:102A1000FF920F931F93CF93DF938C01F62ED72F46
:102A2000C42F222349F081E0809321020E9460207C
:102A30009093200280931F02809121028823C1F08D
:102A400080911F02909120020E947820059780F0CB
:102A5000EF2DFD2FD8014C2F50E0CD01801B910BA5
:102A6000841795071CF48D918193F7CF1092210262
:102A7000DF91CF911F910F91FF9008950E94D22076
:102A80000E9412110C94E3200E94FE1F0E94C2209B
:102A90000E9402110E943E150E94F1200E940A111C
:102AA000FBCF8091280280FF06C06091090170E091
:102AB000660F771F26C081FF04C06091090184E082
:102AC00005C082FF07C06091090188E0689FB001DE
:102AD000112417C0909127029923D1F06091080129
:102AE000961788F72091090188E0289F900111240A
:102AF000929FA001939F500D112470E0CA010E9483
:102B0000EF236038710540F46115710519F406C0B2
:102B100068E070E0862F08958FE7089581E00895BA
:102B20008091280280FF08C06091050170E07595D2
:102B300067957595679521C081FF06C06091050175
:102B400070E07595679519C082FF04C0609105011A
:102B500070E010C090912602992399F060910401D1
:102B60009617A0F780910501899FC001112470E09C
:102B70000E94EF236038710540F46115710519F466
:102B800006C061E070E0862F08958FE7089581E028
:102B900008958D3E21F40E945115819504C08E3E0A
:102BA00029F40E94511580932C0208958F3E21F440
:102BB0000E945115819504C0803F29F40E9451154F
:102BC00080932B020895893F19F40E94901505C047
:102BD0008A3F31F40E949015819580932D020895CB
:102BE0008B3F21F40E949015819504C08C3F29F4FD
:102BF0000E94901580932E0208959FE0980F9830C0
:102C000078F421E030E0A90102C0440F551F9A95E5
:102C1000E2F7CA0190912A02892B80932A02089533
:102C20008D3F21F48091280281600BC08E3F21F4FA
:102C300080912802826005C08F3F29F4809128028C
:102C400084608093280208958D3E39F490912C027F
:102C500097FF35C010922C0259C08E3E29F49091F6
:102C60002C021916BCF32BC090912B028F3E29F435
:102C700097FF25C010922B0249C0803F19F4191606
:102C8000CCF31DC090912D02893F29F41916BCF494
:102C900010922D023BC08A3F19F497FF10C0F8CF65
:102CA0008B3F39F490912E0297FF09C010922E02AB
:102CB0002DC08C3F21F490912E021916BCF39FE099
:102CC000980F983080F421E030E0A90102C0440F51
:102CD000551F9A95E2F7CA01809590912A0289239F
:102CE00080932A0213C08D3F21F4809128028E7FA9
:102CF0000BC08E3F21F4809128028D7F05C08F3F4D
:102D000029F4809128028B7F8093280280912B02E6
:102D1000811106C080912C02811102C010922702FD
:102D200080912D02811106C080912E02811102C076
:102D30001092260208950E94602020912B022111FA
:102D400004C020912C02222321F09093250280932D
:102D5000240220912D02211104C020912E02222351
:102D600021F0909323028093220289E292E00C9456
:102D7000581FEF92FF920F931F93CF93DF9300D0D2
:102D800000D000D0CDB7DEB786E0E9E2F2E0DE01A8
:102D9000119601900D928A95E1F7E0902B02F09048
:102DA0002C0200912D0210912E0210922B021092F3
:102DB0002C0210922D0210922E02E11003C0FF206F
:102DC00009F45DC080912402909125020E94782030
:102DD000AC0190912702992339F020910A0130E04B
:102DE0002417350758F04BC020910B018AE0289F2B
:102DF000900111242417350718F041C09F3F19F0A6
:102E00009F5F90932702EE2061F00E9451151E14DF
:102E100014F09FEF01C091E0989F902D11249093A2
:102E20002B02FF2061F00E9451151F1414F09FEF38
:102E300001C091E0989F902D112490932C02309125
:102E40002B023323E1F020912C022223C1F045EB29
:102E50003403C0011124992319F090932B0203C06D
:102E600081E080932B0235EB2303C00111249923C9
:102E700019F090932C0203C081E080932C02011181
:102E800003C0112309F45DC08091220290912302B6
:102E90000E947820AC0190912602992339F020916C
:102EA000060130E02417350758F04BC02091070188
:102EB0008AE0289F900111242417350718F041C09B
:102EC0009F3F19F09F5F90932602002361F00E94BC
:102ED0009015101614F09FEF01C091E0989F902D6F
:102EE000112490932D02112361F00E949015111668
:102EF00014F09FEF01C091E0989F902D11249093C2
:102F00002E0230912D023323E1F020912E02222354
:102F1000C1F045EB3403C0011124992319F09093BB
:102F20002D0203C081E080932D0235EB2303C00105
:102F30001124992319F090932E0203C081E080930D
:102F40002E0280912B0281110BC080912C028111E5
:102F500007C080912D02811103C080912E02811142
:102F60000E949B16EB82FC820D831E8386E0FE018D
:102F70003196A9E2B2E001900D928A95E1F726968A
:102F80000FB6F894DEBF0FBECDBFDF91CF911F917A
:102F90000F91FF90EF900895E9E2F2E086E0DF0103
:102FA0001D928A95E9F7109227021092260210923C
:102FB00028020895EF92FF920F931F93CF93DF9310
:102FC000EC017B0164E670E088E70E942E1E8C0114
:102FD000EC0EFD1ECE15DF0561F017FD0AC0FE01E7
:102FE000849164E670E00E94AF1E8C012196892BCB
:102FF00089F30E94331FC801DF91CF911F910F9178
:10300000FF90EF90089508950C940318E5E1F3E024
:1030100080E092E0DF019C011D9221503040E1F7F9
:10302000F0931A05E09319058FEF9FEF90935B02E1
:1030300080935A0208950E9404180E9403188093F6
:10304000560280FD02C080E801C080E280935502F4
:103050000E94281E6DE070E08DEC90E00E94DA176F
:10306000892B11F080E008958091560263E070E0B2
:1030700081FD03C08AEC90E002C087EC90E00E94E2
:10308000DA17892B79F76DE070E08AEB90E00E9407
:10309000DA17892B39F70E946C20DC01CB01805AAA
:1030A0009541AF4FBF4F8093150590931605A093A0
:1030B0001705B09318050E94061881E08093590205
:1030C000809358021092570208952091550236E0DD
:1030D000839FC0011124629F800D911D11248115D1
:1030E00022E0920714F080E090E08B5E9C4F90937A
:1030F0001A058093190508952091190530911A0534
:103100002F50334040915502642F70E0C9010E9456
:10311000DB23481B463010F4240F311D211582E0BB
:10312000380710F020E030E02B5E3C4F30931A055A
:10313000209319050895CF93DF938A3011F481E02D
:1031400003C08D3029F480E0DF91CF910C941119E8
:10315000C62F682F8091190590911A0526E0FC0171
:10316000AFE2B2E001900D922A95E1F7603E30F0B7
:1031700026E0FC0111922A95E9F70AC0F6E06F9F5C
:10318000B001112466527F4F46E050E00E940924AE
:10319000C11135C0C0911905D0911A0546E050E023
:1031A000BE018FE292E00E941224892BB1F1C55139
:1031B000D3409E0185E0369527958A95E1F781E019
:1031C00090E0AC0102C0440F551F2A95E2F7209110
:1031D0005A0230915B02242B352B259645E0D6957B
:1031E000C7954A95E1F702C0880F991FCA95E2F783
:1031F000822B932B90935B0280935A020EC0E09136
:103200001905F0911A059F012A5F3F4F2E173F07BE
:1032100009F2808180958193F9CFDF91CF910C9451
:103220007C18CF93E82F2091190530911A0525516C
:10323000334040915502642F70E0C9010E94DB23A6
:10324000481B842FEE2359F066E00E94CF23C82F3D
:10325000C150B0F060E080E20E949B18F9CFA90154
:10326000480F511D4115524018F080E020E030E039
:10327000280F311D2B5E3C4F30931A052093190502
:10328000CF9108951F93CF93DF93EC01162FFE018A
:103290008491882329F0612F0E949B182196F7CFF3
:1032A000DF91CF911F9108950E94421981E00C9403
:1032B0001119809159028823F9F00E946C20DC01D9
:1032C000CB01805A9541AF4FBF4F80931505909326
:1032D0001605A0931705B093180580915802811127
:1032E0000BC062E070E088EB90E00E94DA17892B57
:1032F00019F481E0809358028091580208956F92EA
:103300007F928F929F92AF92BF92CF92DF92EF9275
:10331000FF920F931F93CF93DF93809159028823DD
:1033200009F4DCC020915A0230915B02211531056D
:1033300009F4D4C0809157028111D0C061E070E0DF
:10334000082F10E03B01082E02C0660C771C0A947F
:10335000E2F7A90146215721452B11F48F5FF0CFE9
:1033600090915602980165E0220F331F6A95E1F7AC
:1033700090FD12C08295880F807680930E01220FF7
:10338000232F221F330B319520931101815E8093EF
:103390000F011092120112C045E0369527954A950B
:1033A000E1F7220F220F220F20930E01109211013C
:1033B000295F20930F0183E08093120124E630E01F
:1033C00047E050E06CE071E088E70E94DF1E892B47
:1033D00009F084C08091560280FD23C0A80195E0C9
:1033E000440F551F9A95E1F74B5E5C4F04E610E0E1
:1033F00020E230E060E488E70E94061F892B09F094
:103400006DC00E945919E301C095D09580915A0270
:1034100090915B02C823D923D0935B02C0935A02D8
:103420005DC080E2E5E3F2E0DF011D928A95E9F7F5
:1034300085E0000F111F8A95E1F7AFE8B1E04BE896
:1034400051E0992493942D91EA018991AE01B8013C
:10345000680F711D6B5E7C4F30E02B5C3D4FF901B6
:1034600097E07F01E21AF30AA92C01C0AA0CEA94A2
:10347000EAF77B01B12CE70189917E018A21892E2F
:103480008B18D82DD770CD2E0D2E000CDD08C82F2F
:1034900001C0CC0FDA95EAF7D194C194D108D7E0F6
:1034A000CD22DD2401C08695CA94EAF78C2BD0800A
:1034B0008D298083B39488E0B812DDCF9150319686
:1034C0009F3F79F6C1E0A339BC0709F0BCCF04E601
:1034D00010E020E230E045E352E08CCFDF91CF9165
:1034E0001F910F91FF90EF90DF90CF90BF90AF9022
:1034F0009F908F907F906F90089580915902909146
:103500005802882389F0992369F062E070E086EB25
:1035100090E00E94DA17892B19F0809158020895E3
:10352000109258029091580281E0892708950C94D6
:1035300027050F931F9380915902882329F160E09A
:1035400080E00E9465180E94971A0E947F1980915E
:1035500058028823C9F00E946C2000911505109133
:1035600016052091170530911805DC01CB01801B51
:10357000910BA20BB30B8F3F9F4FAF4FBF4720F470
:103580001F910F910C947D1A1F910F910895CF9365
:10359000DF93EC01FB018281882309F43CC1C43034
:1035A000FDE5DF0760F4CB3F9CE5D90788F49E0179
:1035B00022503C452431310508F02EC109C0C236E5
:1035C000EDE5DE0729F0C63AFDE5DF0709F024C185
:1035D0000E942F1090930C0380930B03C1318CE554
:1035E000D80709F4C6C008F042C0C930ECE5DE07D0
:1035F00009F49BC000F5C5308CE5D80709F485C0F7
:1036000078F4C330ECE5DE0709F478C008F07AC03E
:10361000C230DC4509F0F5C080910B038160EFC03A
:10362000C7309CE5D90709F478C008F07AC08091CA
:103630000B038061E4C0CD30FCE5DF0709F487C0EF
:1036400058F4CB309CE5D90709F479C008F07BC069
:1036500080910B0388606FC0CF30FCE5DF0709F471
:1036600080C008F082C080910B03877FC8C0CE3F26
:103670009CE5D90709F471C000F5C531FCE5DF0709
:1036800009F485C068F4C3319CE5D90709F475C015
:1036900008F095C00E94E20980910B038F77AFC0BC
:1036A000CC3FFCE5DF07A9F108F054C0CB3FDC4577
:1036B00009F0A7C080910C0340C0C230EDE5DE07E1
:1036C00009F489C058F4C1158DE5D80709F45AC02A
:1036D00008F069C080910C0382602FC0C236EDE50E
:1036E000DE0709F47CC0C63AFDE5DF0709F481C0B6
:1036F000C330DD4509F085C080E06EC080910B03CA
:1037000082607DC080910B0316C080910B0388609E
:1037100076C080910C0382604FC080910B03806261
:103720006EC080910B0380646AC00E94E2098091A0
:103730000B03806864C0846062C081603DC080917A
:103740000B038E7F5CC080910B038D7F58C08091EE
:103750000B0316C080910C0318C080910C038D7F61
:103760002BC080910B038F7E4AC080910B038F7D0D
:1037700046C080910B038F7B42C080910B03877FF3
:103780008B7F3DC080910C038D7F8E7F15C0809113
:103790000B0382FB222720F991E0922790FB82F90C
:1037A00090FB83F92CC080910C03982F9095917019
:1037B0008E7F892B90FB81F980930C0322C00E949D
:1037C000E20980910B0387FB222720F991E09227E1
:1037D00090FB87F914C081E00E94C61012C080914E
:1037E0000B0384FB222720F991E0922790FB84F9B8
:1037F00006C080910B03982F909590FB80F98093E1
:103800000B0380910B0390910C030E9440100E94C7
:10381000E20980E001C081E0DF91CF9108958FE857
:1038200091E00197F1F700C0000008950C942E0577
:10383000EF92FF920F931F93CF93DF93C7EAD1E0EC
:1038400003EA11E09801DE0141E050E081E0AB3A8B
:10385000B80769F18D91E82FE295EF70F0E061A172
:103860008F707A0102C0EE0CFF1C8A95E2F7C70147
:103870009E2D9095962391A392A1892B82A3F90165
:1038800081919F01E82FE295EF70F0E061A18F70C8
:103890007A0102C0EE0CFF1C8A95E2F7C7019E2D4B
:1038A0009095962391A392A1892B82A3CFCF0E94BA
:1038B0000F1CE4E6F2E0B2E0E836FB0739F12991AB
:1038C000A22FA295AF70B0E090968C9190E02F70EF
:1038D00002C0959587952A95E2F78170D8019D9150
:1038E0008D01A92FA295AF70B0E090962C9130E099
:1038F0009F7002C0359527959A95E2F720FD02C08A
:1039000090E001C092E0892B8193D5CFDF91CF91D8
:103910001F910F91FF90EF9008952F923F924F9239
:103920005F926F927F928F929F92AF92BF92CF924F
:10393000DF92EF92FF920F931F93CF93DF9384E672
:10394000682E82E0782E97EAE92E91E0F92E03EABC
:1039500011E020E6822E22E0922ECCE5D2E0630137
:103960005301312C212C34E0432E512CD501ED9103
:103970005D014E2F440F440FF60141936F01D701B3
:103980002D917D01E22FE295EF70F0E080A190E0B3
:103990002F7002C0959587952A95E2F78170992737
:1039A000F80151918F01E52FE295EF70F0E020A131
:1039B00030E05F7002C0359527955A95E2F7F9011E
:1039C000E170FF2720FF02C0E2E0F0E0E82BF92BD6
:1039D000E42BD301ED933D01EF70F0E0ED56FE4F87
:1039E0009081F4018081890F808384304CF088813C
:1039F0008F5F888360E0832D0E94161C21E001C048
:103A000020E0D4018C918D3F44F4888181508883DB
:103A100061E0832D0E94161C21E0F4018081082EB4
:103A2000000C990BB2010E94EF23D4018D934D013C
:103A3000222A33942196B4E03B1298CF822DDF9155
:103A4000CF911F910F91FF90EF90DF90CF90BF909B
:103A5000AF909F908F907F906F905F904F903F902E
:103A60002F900895CF93DF9386319C4541F5EB016C
:103A70000E94330F982F8A81209102013091030117
:103A8000882379F09A7A81E009F480E080936802D3
:103A9000911102C069E201C065E3C9010E94D41F0F
:103AA0000AC080916802811102C069E201C065E329
:103AB000C9010E94D61F0E94750F80E001C081E0FD
:103AC000DF91CF9108950F931F93CF93DF93C42F6E
:103AD000D22FFC0182818823C9F040936B020E949F
:103AE000602090936A028093690280E28C0F883094
:103AF00008F057C0C77081E001C0880FCA95EAF787
:103B0000DF91CF911F910F910C94300780916B0240
:103B1000481330C08091690290916A020E94782017
:103B2000883C910538F510E21D0FCD17B9F080E201
:103B30008C0F883040F4C77081E001C0880FCA95AF
:103B4000EAF70E943707183028F581E09D2F97701B
:103B500001C0880F9A95EAF70E943007802F0E94D3
:103B600027071830F0F4D77081E001C0880FDA958C
:103B7000EAF70AC080E28C0F883098F4C77081E0C1
:103B800001C0880FCA95EAF7DF91CF911F910F917D
:103B90000C943707802FDF91CF911F910F910C94D8
:103BA0002707DF91CF911F910F9108950F939C01EB
:103BB000CB01243F4CE5340731F188F4293DFCE585
:103BC0003F07D9F02A3D4CE5340779F1283D3C45C3
:103BD000A9F506E221EE41EE68ED7CE52BC0263F1B
:103BE000FCE53F07E1F0A8F0273F3C4539F507E247
:103BF00025EE46EE67EF7CE51DC007E225EE45EEBB
:103C000069ED7CE517C006E221EE40EE64EF7CE54D
:103C100011C007E225EE44EE65EF7CE50BC006E23D
:103C200021EE42EE66EF7CE505C008E221E045EEBC
:103C30006AED7CE50E94631D80E008C0FC01828182
:103C4000882319F010926B0201C081E00F91089552
:103C50001092B9008CE08093B80008959F92AF92C3
:103C6000BF92CF92DF92EF92FF920F931F93CF9369
:103C7000DF93B82EEB010E9460206C01C431D105A6
:103C800058F0CF3F8FEFD80759F0CE0164E170E0D4
:103C90000E94DB237B0107C0EE24E394F12C03C0D8
:103CA00025E0E22EF12C84E8A82E94EA992E1092B9
:103CB000BC009092BC000E9460208C018091BC00EE
:103CC00087FD08C00E946020801B910B8E159F0508
:103CD000A8F32AC08091B900887F883041F0809194
:103CE000B900887F803119F00FEF1FEF1FC0B0922D
:103CF000BB00A092BC000E9460208C018091BC009F
:103D000087FD08C00E946020801B910B8E159F05C7
:103D1000A8F30AC08091B900887F883111F08034FF
:103D200019F700E010E00EC00EEF1FEFCF3F8FEF4E
:103D3000D80709F4BCCFC6010E9478208C179D07D4
:103D400008F4B5CFC801DF91CF911F910F91FF907B
:103D5000EF90DF90CF90BF90AF909F9008950F931A
:103D60001F93CF93DF93EB018093BB0084E8809394
:103D7000BC000E9460208C018091BC0087FD0EC0B9
:103D8000CF3F8FEFD807C1F30E946020801B910BBB
:103D90008C179D0788F38EEF9FEF0CC02091B90020
:103DA000287F81E090E0283211F480E090E0919546
:103DB00081959109DF91CF911F910F910895CF9235
:103DC000DF92EF92FF920F931F93CF93DF936B01DC
:103DD0008A017901B9010E942E1EE6010C0D1D1DFC
:103DE000C017D10761F424E92093BC00DF91CF9183
:103DF0001F910F91FF90EF90DF90CF90089597FD66
:103E0000F2CFB70189910E94AF1EEACFCF92DF9225
:103E1000EF92FF920F931F93CF93DF93C62F6A0108
:103E20007901B8010E942E1E97FD11C0B8018C2F98
:103E30000E94AF1EE601EC0CFD1CCE15DF0539F02B
:103E400097FD05C0B80189910E94AF1EF6CF24E905
:103E50002093BC00DF91CF911F910F91FF90EF90C5
:103E6000DF90CF90089584E98093BC0008959093EB
:103E7000AD018093AC01089590937102809370021C
:103E80000895E0917002F0917102309721F0019055
:103E9000F081E02D099480E00895E0917002F091A6
:103EA0007102309721F00280F381E02D099408958A
:103EB000E0917002F0917102309739F022E0DC015C
:103EC0002C930480F581E02D0994089520916E02D1
:103ED00030916F022817390771F090936F02809329
:103EE0006E02E0917002F0917102309721F006802D
:103EF000F781E02D0994089520916C0230916D02B4
:103F00002817390771F090936D0280936C02E0914D
:103F10007002F0917102309721F00084F185E02D5C
:103F200009940895FC01329697E080E0915029F0C1
:103F300021912223D9F38F5FF9CF0895662349F0A9
:103F4000FC01329608962191621729F0E817F907CB
:103F5000D1F780E0089581E008959C01FC0132963C
:103F60009FEF80E04191461789F09F3F19F441117E
:103F700001C0982F8F5F8630A9F79F3F39F0F90174
:103F8000E90FF11D97FDFA956283089508959C014C
:103F90002A5F3F4FFC014281461301C01282019605
:103FA00082179307B9F708950C94AD1F0C94C71F9F
:103FB000029626E0FC0111922A95E9F708950895EA
:103FC0000C94DF1F0C94E01F0C94DF1F0C94DF1F78
:103FD0000C94DF1FCF930E94E61F0E94C5140E941D
:103FE000E41FC0E08C2F0E94FD13811104C0CF5F3D
:103FF000C430C1F701C081E0CF91089508951F92A8
:104000000F920FB60F9211248F939F93AF93BF938C
:1040100080917202811113C080911B0590911C0543
:10402000A0911D05B0911E054196A11DB11D809363
:104030001B0590931C05A0931D05B0931E05BF9111
:10404000AF919F918F910F900FBE0F901F90189579
:1040500080917502882331F10E9409061092720244
:1040600020E488E190E00FB6F894A8958093600072
:104070000FBE2093600083B7817F846083BF83B7C6
:10408000816083BF7894889583B78E7F83BF0FB696
:10409000F894A895809160008861809360001092E8
:1040A00060000FBE08950E94E2090C940F0682E0A2
:1040B00084BD93E095BD9AEF97BD80936E000895FF
:1040C0002FB7F89480911B0590911C05A0911D05B8
:1040D000B0911E052FBF08952FB7F89460911B056E
:1040E00070911C0580911D0590911E052FBF0895AC
:1040F0009C014FB7F89480911B0590911C05A091ED
:104100001D05B0911E054FBF821B930B0895789437
:104110001F920F920FB60F9211248F939F93AF931C
:10412000BF9380911B0590911C05A0911D05B09136
:104130001E050196A11DB11D80931B0590931C05C2
:10414000A0931D05B0931E05BF91AF919F918F91D4
:104150000F900FBE0F901F90189598E088E10FB652
:10416000F894A895809360000FBE90936000A89586
:10417000F894D8E0CEEF28E3299320E0299314BEE9
:10418000FFCF08950E946020909374028093730281
:1041900090E080E80FB6F8948093610090936100FE
:1041A0000FBE08950E94B423539A80E0815041F0DD
:1041B000A895EFE9FFE03197F1F700C00000F6CFD6
:1041C0005398789408950E94D7210E943C1F2FEFA6
:1041D00080E792E0215080409040E1F700C000006D
:1041E000089580914605882389F0109246050E9423
:1041F00060209093740280937302809175028823EB
:10420000D1F1109275020E94532011C08091750265
:10421000811111C080917302909174020E947820E4
:10422000069728F081E0809375020E9428208091F3
:104230007502882301F10E9428200E94EA1F88232A
:1042400039F1F8942AB15B9A822F8C608AB99BB1BC
:104250008CE098279BB93FE748E391E0315040401C
:104260009040E1F700C000009BB189278BB92AB9C3
:104270005B98789408950E94BD2280914C05882314
:1042800029F080912A0584FD0E94A5110C947E21BD
:10429000089580910A030895089590917B029813E0
:1042A00007C02091790230917A0226173707A9F0CA
:1042B00080937B0270937A026093790280937602F6
:1042C00070937802609377028091630584FF05C044
:1042D00063E086E792E00C94B9220895BC0184E083
:1042E0000C944D21BC0183E00C944D212091630579
:1042F00024FF03C066E00C94B9220895CF93DF93A6
:10430000CAE0D0E080912A0584FF18C0809187021E
:10431000909188029817E1F028E0829FC001112453
:1043200068E087579D4F0E94B5228091870290E0F8
:1043300001968F709927809387020AC00E94BD2240
:104340008FE99FE00197F1F700C000002197D1F6B7
:10435000DF91CF910895CF93DF93EC01A091880274
:10436000B0E0CD0101968F70992720918702281720
:1043700079F093E0AA0FBB1F9A95E1F7A757BD4FBD
:1043800098E0FE0101900D929A95E1F780938802E2
:104390000E94BD220E947E2188E0FE01AFE7B2E0CC
:1043A00001900D928A95E1F7DF91CF91089583E115
:1043B00091E00895FC01808180768032A1F58181B1
:1043C000813061F484819581892B69F58FE792E0D2
:1043D000909348058093470588E00895823041F422
:1043E00089E093E0909348058093470581E0089524
:1043F0008A3021F483818093090315C0893099F4B0
:10440000828193818115924081F484819581892BE9
:1044100061F481E080937E028681978190937D0292
:1044200080937C0202C080E008958FEF0895209170
:104430007C0230917D02232B71F020917E0221308D
:1044400051F4FC01808180930A0310927D02109246
:104450007C0281E008958FEF08950895FC01938117
:104460009330D9F068F4913081F0923009F059C05E
:104470008AE196E090934805809347058BE3089581
:10448000913249F19232B9F14CC085E596E09093B2
:1044900048058093470582E108958281813099F033
:1044A00050F08230F1F587E696E0909348058093CE
:1044B00047058EE108958DE996E090934805809335
:1044C000470584E0089587E896E090934805809337
:1044D000470584E108958281882329F0813009F518
:1044E00085E496E002C08CE296E0909348058093C4
:1044F000470589E0089584819581009751F00197DF
:1045000081F481EA96E090934805809347058BE714
:1045100008958CE197E0909348058093470580E4E7
:10452000089580E008951F93CF93DF93162FEA013B
:10453000288124FF05C0398128E82327298302C068
:104540002AE52883212FFC01CE010296DC0131915E
:104550003D9321501216DCF3612F0E94E2031C5F91
:104560001883DF91CF911F9108954AE255E00C9492
:10457000932243E655E00C949322CF93DF9360910E
:104580004905635067FD93C080914505CCE0D0E0BC
:10459000C81BD109C35BDA4F80914405803120F4F8
:1045A000CE010E942D2281C08D3209F06EC068308C
:1045B00009F07BC083EC80931F058AE5809320017E
:1045C000109243058881807621F0CE010E94DA2185
:1045D00049C09A81109228058981811106C01092E4
:1045E000290528E235E082E038C0853019F490933F
:1045F0004A0530C08630A1F48B81813041F0823091
:1046000031F0833021F0813211F0823221F4CE0179
:104610000E942E2201C080E090E49093430522C0C6
:10462000883089F0893019F490934C0513C08A3092
:1046300069F08B3079F48BE480932B0580936405CB
:104640008093370507C02CE435E002C028E235E04E
:1046500081E003C028E235E080E0309348052093F4
:10466000470509C08F3F39F4988197FD8E8190E806
:104670009093430507C09F81911104C09E819817B4
:1046800008F4892F80931F0110C08091430587FF94
:104690000CC0CE010E9417228F3F21F48EE180933F
:1046A000200103C0811110921F01109249058091D1
:1046B000200184FF4CC080911F018F3F09F447C047
:1046C000C82F893008F0C8E08C1B80931F0190919F
:1046D0001F0588E8892780931F05CC2359F1809115
:1046E0004705909148052091430526FF12C0AFE190
:1046F000B5E02C2FAC014F515540FA01EA0FFB1FDA
:10470000E4911196EC931197215011962111F5CF58
:1047100008C0E0E2F5E0DC012C2F3D9131932150FF
:10472000E1F701962FEF2C0F820F911D9093480512
:10473000809347056C2F80E295E00E94E203CC5FF6
:10474000CC3019F08FEF80931F01C093200184E1DA
:1047500099B19C7031F48150D9F710924A051092AA
:104760004205DF91CF910895CF93DF93E9E6F0E022
:10477000808188608083E99ACAE2D5E08BE48983EE
:10478000A3E6B5E011968C931197E6E3F5E08183FB
:104790008AE588838C938083DF91CF910895991B5C
:1047A00079E004C0991F961708F0961B881F7A9528
:1047B000C9F780950895AA1BBB1B51E107C0AA1F2A
:1047C000BB1FA617B70710F0A61BB70B881F991FB2
:1047D0005A95A9F780959095BC01CD01089597FB56
:1047E000072E16F4009407D077FD09D00E94DB2332
:1047F00007FC05D03EF4909581959F4F08957095E4
:1048000061957F4F0895EE0FFF1F0590F491E02D05
:104810000994FB01DC0102C005900D92415050400B
:10482000D8F70895FB01DC0104C08D910190801937
:1048300021F441505040C8F7881B990B0895F9990D
:10484000FECF92BD81BDF89A992780B50895A8E161
:10485000B0E042E050E00C945324262FF999FECFAB
:1048600092BD81BDF89A019700B4021639F01FBAC3
:1048700020BD0FB6F894FA9AF99A0FBE08950396E0
:10488000272F0E942E240E942D24252F0E942E24A3
:10489000242F0C942E240196272F0E942E240C9452
:1048A0002D24DC01CB01FC01F999FECF06C0F2BD3D
:1048B000E1BDF89A319600B40D9241505040B8F7DE
:0648C0000895F894FFCFFB
:1048C600C8000402280850011E0A14010021007FB6
:1048D6002200034921AB21762172216E214C21FF52
:1048E6005AE200E900EA00B500B600B700CD008341
:1048F60001CC008A0192019401210223022402259F
:1049060002260227022A02B300B4006F007000815B
:104916008283E200E900EA00B500B600B700CD00E8
:104926008301CC008A019201940121022302240210
:104936002502260227022A02B300B4006F00700087
:10494600818283309796956061626300081018181B
:1049560010080000FF0100010000FFFF0000010039
:0C49660001FF0090313335913234940091
:00000001FF
